:020000040000FA
:020000002128B5
:08000800A000030E8301A1001A
:100010000408A2000B1D1A280B11230832208600A9
:10002000A30A203023020319A301831681110111B1
:100030000110831222088400210E8300A00E200EDE
:1000400009008601831686018312AA308600A30167
:100050008B170B118316811281110111011083126C
:100060008B163128820789340034893489347634F8
:1000700000347634893489340034893400340034CF
:1000800000340034003400340034003400340034D0
:1000900000340034003400340034003400340034C0
:0600A000003400340034BE
:02400E00F13F80
:00000001FF
